:020000020000FC
:10000000A7CDA5C10000000020C0000089C00000ED
:10001000000093C00000000000000000020304067E
:10002000080C10182030406080000406080C1018DE
:100030002030406080A0C0000003070F1F000D0D9E
:1000400004050D050205030302004FB662FD0CC056
:10005000552041F00994C52DC095089483FDC7959E
:10006000C4BD64604FBE1895C0916400089483FDC0
:10007000C795C4BD6B7FC0916400CF3F09F419C020
:100080004FBE9198909893981895919890989398BE
:1000900076FD0DC065FD0BC0C9E0CA95F1F7C091B2
:1000A000B100C0FD949AC1FD979AC2FD959A4FBECA
:1000B000189524BCCC27C064C8BF6460F8CFCBCFF0
:1000C00070FFC9CF65FDC7CF919AC5CF70FFC3CF71
:1000D00065FDC1CF909ABFCF70FFBDCF65FDBBCF8F
:1000E000939AB9CF949870FFB6CF65FDB4CFCEE1A7
:1000F000CA95F1F7919AAFCF979870FFACCF65FD95
:10010000AACFCEE1CA95F1F7909AA5CF959870FF46
:10011000A2CF65FDA0CFCEE1CA95F1F7939A9BCF10
:100120004FB6C9B7CF7EC9BF6E7FCCB5CE0DDDB59A
:10013000DF1DDBBDCABD4FBE18953FB68F7EABB786
:10014000A074A2118061A0E0ABBFA9B7AE7FA9BF28
:100150007894A0916800AA2341F085FD2AC0A0915F
:100160006800AA95A093680024C040E050E085FD97
:1001700014C0A0B396FFA095A2FD4FEFA3E096FF99
:10018000A2E0A5BFAA27A064AABF8D7FA0B396FF57
:10019000A095A2FD5FEF451741F7A8E161FDA0938F
:1001A000680085FD03C0A8E1A09368004093960015
:1001B000816085FD0EC0A0916900AA2331F0A09155
:1001C0006900AA95A093690004C08061AA27A06471
:1001D000AABF80FF3CC0A09196004A2F61FF8E7F8E
:1001E00085FD1CC0A091B400A430C1F4403F08F0CC
:1001F00040EFA42FA295AF704A0F5091B600533034
:1002000069F0A695A69550FD01C0A69552FD03C0C4
:10021000A41B4A2F03C04A0F08F44FEF409361001C
:10022000A72FA670A1F073FD12C0A0917000AA0FB5
:10023000AA0F50919E0056955695541708F0452FD9
:100240004A0F4093610018F4AFEFA0936100409112
:10025000B400443009F03AC0A0916100A09363005B
:1002600040916300A0919B004A1708F04A2FA0918B
:100270009D004A1708F04A2F542EA091A000AA23EF
:1002800009F422C0542F5A1B10F4A42F50E0BA2EA8
:100290008894AA1FAA2EA091A200A095AA22A50E1A
:1002A00058F0A091A100A21509F0AA95AA0EA0935A
:1002B000A10048F04A2D08C0A091A100BA1608F08C
:1002C000A395A093A1004FEF40936400A52DA03407
:1002D00008F06860A0916000A395A093600051F0C1
:1002E000F894A9B7A160A9BF84FF02C0A0E4ABBF86
:1002F0003FBE1895A0917400A395A093740041E0AF
:1003000050916800552329F085FF03C05A955093FA
:100310006800A0919600A13018F0209299000DC0BD
:1003200020929A002092A300A0919900AF5FA09321
:10033000990018F0AFEFA0939900F894A9B7A160C5
:10034000A9BF84FF02C0A0E4ABBF3FBE18953FB673
:100350004CB55DB58F7EABB7A074A2118061A0E0F3
:10036000ABBFA9B7AE7FA9BF789481FD23C0A2E03F
:1003700096FFA3E0A5BF8260A0B396FFA095A2FF61
:1003800005C040936500509366003EC1A3E096FF10
:10039000A2E0A5BFAA27A064AABF8D7F85FF01C0E8
:1003A00026C140E0A0B396FFA095A2FD20C14093D6
:1003B00096000FC1A3E096FFA2E0A5BF8D7F61FF6D
:1003C00071C0A2E096FFA3E0A5BFAA27A064AABFC0
:1003D00082604093910050939200A0908F004A1940
:1003E000B09090005B09BB24A22C4C38520518F445
:1003F0002092950049C0A091D400AA2359F1483C0D
:10040000520528F4A0E1BA2EAAE0AA2E23C048364D
:10041000A1E05A0728F4A8E0BA2EAFE0AA2E1AC02D
:10042000403DA2E05A0728F4A4E0BA2EAEE1AA2E7D
:1004300011C0403AA5E05A0728F4A2E0BA2EACE376
:10044000AA2E08C04839A8E05A0720F4A1E0BA2E25
:10045000A8E7AA2EC42EA0919300CA1AD52EA09167
:100460009400DA0ADD202AF4AFEFC094D094CA1ABF
:10047000DA0A20929500A8E0A210A0E0CA14DA06D9
:1004800018F4A1E0A093950040939300509394003A
:10049000409191005091920040938F0050939000B2
:1004A00042E097C0A09165004A1BA09166005A0BDC
:1004B00094FD82C093FD80C092FD7CC086FF03C086
:1004C000D52EC42E0CC05695479591FD73C05695F8
:1004D000479590FD6FC0D52EC42ED694C79461FD6C
:1004E00019C0AC2DAC51AD2DA24008F005C0DD20E7
:1004F00089F4AC2DA85C70F4A0916700A395AA23A1
:1005000011F0A0936700AA3008F471C02092960001
:1005100081606DC0A0916700AA2319F0AA95A093ED
:100520006700A22C5091BA0097FD06C0A090C800A9
:10053000533011F4A090D000AAEFAA0EA22DA21D54
:10054000CA18DA0A4FB74170533049F4442321F0F6
:1005500087FD05C0806803C087FF01C08F774423F3
:1005600059F0533031F4AFEFC094D094CA1ADA0A7C
:1005700003C040E050E020C0533049F4CC0CDD1CF7
:10058000AAE0CA1AD20818F4A0E0CA2ED22CAFEF03
:10059000CA16D20418F04FEF50E00EC0A091AC0084
:1005A000CA9E412D000C441F50E008F012C04FEFCE
:1005B00050E00FC05695479594FF07C0552309F0AA
:1005C0004FEFA42FA6954A0F521D4F3F520508F03A
:1005D0004FEF40939600816061FF09C0AFE1A095A5
:1005E000A923AB299A2F8F7DBB2009F48062A8E153
:1005F000A093680085FF03C0AAE0A093680061FD96
:1006000003C085FD01C08F7E85FD03C0A6E0A093D9
:100610006900F894A9B7A160A9BF84FF02C0A0E453
:10062000ABBF3FBE189511E00AC013E008C01AE046
:1006300006C01EE104C014E602C018EC00C005E1CB
:10064000BB27BA95F1F70A95D9F71A95C1F708951E
:100650002AE338E709C020E33CE806C02AE234EB8D
:1006600003C025E238EC00C012E0BB279798BA958A
:10067000F1F7909ABA95F1F79098BA95F1F7979AA1
:10068000BA95F1F7123009F0919A123009F4939A61
:10069000B091AD00BA95F1F7123009F0919812308F
:1006A00009F49398B7E8BA95F1F71A95F1F6022F85
:1006B000B22FBA95F1F70A95D9F73A95A9F6979816
:1006C0000895221B39E0001F3A9509F40895221F6E
:1006D000211B18F4210F8894F6CF0894F4CF622CD4
:1006E000722CB0E08894B395221F331FE0F7379542
:1006F00027958894912E802E020B130B10F4192D40
:10070000082D10F4889401C00894661C771CBA95D3
:1007100071F7172D062D0895322D11232AF43A95DD
:1007200000951095031B130BF894029F712C002D5C
:10073000129F912C802C7894780C172D921C292DC7
:10074000B4E06B2E2695179507956A94D9F7332355
:1007500021F000951095031B130B08950091B40030
:100760000430A1F1B0919600B15008F010C0B091E2
:100770006100B093630020927E0020927F0020925F
:10078000800020928100209282006F7B1FC06090C9
:10079000B4006064B0916100B093620008E317ECAC
:1007A00020917A0030917B0036952795B62DBA9529
:1007B00041F036952795B62DBA95BA9511F0369534
:1007C00027958DDF00937E0010937F0008950091A0
:1007D0007E00B09162000B1B10917F00120928F47B
:1007E0000038BFEF1B0740F009C00F37120508F4AF
:1007F00005C00FE710E002C000E81FEF0093830080
:1008000010938400089500918300B09180000B0F35
:1008100010918400B09181001B1F20E03091840072
:1008200033230AF42A95B09182002B1F1AF4203F3B
:1008300040F00AC02F3008F407C00FEF1FEF2FE081
:1008400003C000E010E020EF30916300B0919B0006
:100850003B1718F4323030F009C0B0918400BB234C
:100860005AF004C0B0918400BB2332F4009380009E
:10087000109381002093820008952091D700009169
:100880008300000F10918400111F46DF11232AF40A
:100890000038BFEF1B0740F009C00F37120508F4FE
:1008A00005C00FE710E002C000E81FEF002352F080
:1008B000B0916200B01B0B2F18F0013008F00AC095
:1008C00001E008C000950F5FB09162000B0F08F0C7
:1008D00001C00FEF0093850008952091D80000918A
:1008E00081001091820018DF11232AF40130BFEF3C
:1008F0001B0740F009C00F3F120508F405C00FEFB9
:1009000010E002C001E01FEF112352F0B09185000A
:10091000B01B0B2F18F0013008F00AC001E008C02E
:1009200000950F5FB09185000B0F08F001C00FEF2D
:100930000093630008950FEF677F71FD29C072FD7A
:1009400009C06860B0917B00BA3020F0B52DB0349A
:1009500008F4677FB091D300BB23D1F0B0917B0046
:10096000BB23B1F00FEF10917B00ABDEF894B09198
:10097000730072FDB5E00B9F112D002D78941123AB
:1009800009F00FEFB0919E000B1710F400919E003C
:1009900000939D00089500917A0010917B0000540F
:1009A0001140B0919D0010F4BA9501C0B39511F0BB
:1009B000B0939D00089500C008952091B500B6B190
:1009C000B6FDFBCF04B115B1B6B1BF77B6B9B091E2
:1009D000AA00B395B093AA00B83060F12092AA00A3
:1009E000B091D200BB2321F1112329F0B091AB00CB
:1009F000BF3F61F009C0B091AB000B1739F020F494
:100A0000BB2321F0BA9502C0B395E1F300919B009E
:100A1000B093AB00B03050F400ECB03038F400E8E4
:100A2000B03020F400E4B03008F400E000939B0004
:100A30007F7E089510919B00B0E11B0F08F41FEF1B
:100A400010939B00B091B400B43081F000919B00F2
:100A5000B0916300B01B10F400916300B0919D0051
:100A60000B1708F00B2F502E00936400B091AA00D2
:100A7000B73009F47061089502E3F894B091D90099
:100A80000B9F012D000C001F7894B0919B000B1759
:100A900010F000919B000093610000936300502EC2
:100AA0000093640000939E00089520927A00B0EFB6
:100AB000B0937B000895F8940CB51DB52091740097
:100AC00078943091750060907600009375001093D3
:100AD0007600031B160971FD03C077FD7DC027C09A
:100AE00070907700209377002709222311F00FEFF1
:100AF0001FEF80907800909079003093780060929A
:100B0000790000917500109176000819190920915B
:100B10007A0030917B0036952795020F131F10F451
:100B20000FEF1FEF00937A0010937B0029C02091F4
:100B30007A0030917B003901B4E08B2EB2E09B2E1D
:100B4000343010F08A949A94383010F08A949A9441
:100B5000769467948A94E1F726193709992021F051
:100B6000169507959A94E1F7200F311F20937A008C
:100B700030937B0028F43FEF30937A0030937B0072
:100B8000323008F4706871FF02C0B3E00DC0B0915C
:100B9000C40000917100023838F0B395003A08F0B3
:100BA000B395B63008F0B5E09B2EB4E08B2E1091D3
:100BB0007B0000917A0024E0169507952A95E1F7CD
:100BC0000819120928F0B02FB250B12FB20910F451
:100BD00002E010E0980126C020917A0030917B005D
:100BE000390176946794669466946694261932095E
:100BF00006950695200F321D20937A0030937B00D6
:100C0000323008F07F7704E03695279536952795A2
:100C100026952695201B10F0223008F422E0890149
:100C20009090C40060FDFECFE0908B00F0908C00AF
:100C30006160B9B7B061B9BF380177FD41C0769442
:100C4000679400938B0010938C00B92DB330E1F0C2
:100C5000B0FD04C0060D171D930106C0000F111F43
:100C60000250120922E030E0B92DB33068F0209331
:100C70008D0030938E00009387001093880060925F
:100C8000890070928A003AC000938D0010938E0004
:100C900020938700309388006092890070928A00C8
:100CA00071FF0DC0BFE0B0938D0020928E00B09315
:100CB000890020928A00B0938B0020928C001EC085
:100CC000669400938B00B92DB33091F0B0FD03C052
:100CD000060D262D03C0000F025022E0B92DB330BF
:100CE00038F020938D00009387006092890006C041
:100CF00000938D00209387006092890000917C0012
:100D000002FD0350013031F495FD0CC0B2E0B06C2F
:100D1000B7B90BC0023021F4B3E0B06CB7B905C06D
:100D200095FDF4CFB4E0B06CB7B90091A200000F0C
:100D300010F4BBE60B270093A20060FDFECFB2E0EB
:100D4000B0936E006160B9B7B061B9BFB72FB6702C
:100D5000D1F020917A0030917B0036952795369519
:100D6000279571FF02C0B0E43B0FF8940CB51DB598
:100D7000020F131F1BBD0ABD6160B0E1B8BFB9B758
:100D8000B061B9BF78940895606120927D0020E041
:100D900067FD20E206C0606120927D0020E267FDD1
:100DA00020E001E011E077FD11C0B72FB67009F027
:100DB0006F7E14E100917B00069509F403950F30D6
:100DC00008F00FE071FF02C004E114E160FD0FC004
:100DD000B0917D00BB2359F071FF06C0B0916E0049
:100DE000BA95B0936E0011F4706247C0ABDFB0B734
:100DF000B77FB0BFB8B1B0B7B860B0BFB0917D0039
:100E0000B395B0937D00B8B177FD06C0B1E071FD38
:100E1000B3E0BA95F1F7B8B1B072B21709F022C0D9
:100E200071FF05C00395011708F00A95CFCF64FD47
:100E300005C00395011708F0B4CFC8CF6F7EF894B2
:100E40003CB56DB470907A0080907B00370D681CC3
:100E50006BBC3ABD6160B0E1B8BFB9B7B061B9BFB2
:100E600078949FCFB0916D00B13008F49ACF64FDB3
:100E700098CF0A9509F0AACF7F7D20918D003091FF
:100E80008E00F894B0E1B8BF0CB51DB5020F131F6A
:100E90001BBD0ABDE0908700F09088006160B9B783
:100EA000B061B9BF7894B72FB67039F0B0916D00CA
:100EB00072FFB395B0936D0009C075FF07C067FD61
:100EC00005C064FD03C0BF91BF91EEC4089500E06A
:100ED00063FF03C064FF01C001E0F894109171004A
:100EE000B7E01B9F212D102D7894200F2695179584
:100EF000269517952695179510937100183718F4B5
:100F0000B8E7B093710000917100B09172000B17B7
:100F100020F0606291989098939860FDFECFE090E9
:100F20008900F0908A006160B9B7B061B9BF0895D7
:100F3000B2E095FD0AC0F894B0937C009798949A1B
:100F400062FF01C0939A7894F4C0F894B0937C0047
:100F50009798959A62FF01C0919A7894EAC0B3E09D
:100F600082FF24C095FD11C002E0F894B0937C008C
:100F7000ECE7F0E00093B1009398959862FF02C00F
:100F8000909A01C0979A7894D4C002E0F894B093F4
:100F90007C00ECE7F0E00093B1009198949862FF38
:100FA00002C0909A01C0979A7894C3C095FD0BC077
:100FB000F894B0937C00E6E6F0E0939862FF01C0FD
:100FC000909A7894B6C0F894B0937C00E6E6F0E08E
:100FD000919862FF01C0909A7894ABC0B4E095FDFF
:100FE0000AC0F894B0937C009498959A62FF01C06F
:100FF000909A78949EC0F894B0937C009598949AB7
:1010000062FF01C0909A789494C0B5E082FF24C03A
:1010100095FD11C001E0F894B0937C00E2E7F0E0A8
:101020000093B1009098979862FF02C0919A01C016
:10103000949A78947EC004E0F894B0937C00E6E83B
:10104000F0E00093B1009098979862FF02C0939AE5
:1010500001C0959A78946DC095FD0BC0F894B0933B
:101060007C00E0E6F0E0909862FF01C0919A7894ED
:1010700060C0F894B0937C00ECE6F0E0909862FFDA
:1010800001C0939A789455C0B6E095FD0AC0F894D3
:10109000B0937C009598979A62FF01C0919A7894DA
:1010A00048C0F894B0937C009498979A62FF01C06E
:1010B000939A78943EC0B1E082FF24C095FD11C0A0
:1010C00004E0F894B0937C00E6E8F0E00093B1000F
:1010D0009198949862FF02C0939A01C0959A78946F
:1010E00028C001E0F894B0937C00E2E7F0E00093C0
:1010F000B1009398959862FF02C0919A01C0949AAA
:10110000789417C095FD0BC0F894B0937C00ECE682
:10111000F0E0919862FF01C0939A78940AC0F89425
:10112000B0937C00E0E6F0E0939862FF01C0919AF2
:1011300078946F7D08952FE530E0F9012092B10099
:101140009198909893989498979895986B7F089514
:10115000A2EBB0E009E00D9309E00D9304E00D93DC
:101160000FEF0D9303E00D930FEF0D9309E00D9337
:1011700001E00D9301E00D9301E00D93AEEBB0E0C3
:1011800001E00D930FEF0D930D930D930D930D93C0
:1011900003E00D930FEF0D930FEF0D930D9305E209
:1011A0000D9300ED0D9308E20D9300E50D9304E01F
:1011B0000D930FEF0D9302E00D9300E00D930AE7FE
:1011C0000D930FEF0D9300E00D9301E00D9300E000
:1011D0000D9303E00D9300E00D9308952091B90065
:1011E0008B7FB091BA00B33019F09F7DB1FD906252
:1011F0009F7BB091BB00B1FD9064223011F08860FC
:1012000001C0877F08950A95E00FF21DB4910895FB
:10121000ECE1F0E00091B200F6DFB093D700ECE132
:10122000F0E00091B300EFDFB093D800EAE2F0E025
:101230000091B800E8DFB093D9000091B800023007
:1012400008F402E000937300B091CE000FEFB230CB
:1012500009F400EAB33009F402E800937200E8E30D
:10126000F0E00091D500CFDFB093A000089508957D
:101270002091C8003091C900B091BA00B33009F490
:101280003E5097FF02C020E03FEFB32FB21B6B2E02
:10129000B25810F4B2E86B2E00E00395609EB12DB9
:1012A000BD57D8F30093AC0008959068E1DFC1D931
:1012B00020E030E0B0E16B2EB8D9B09196002B0F52
:1012C000321D6A94C9F7B4E036952795BA95E1F7CF
:1012D000822E9F77CDDF0895F894E3E0F0E0B9E047
:1012E000B7BFB491B078C1F3F894A895B1B5B8611F
:1012F000B1BDB0E0B1BDB4E0BEBFBFE5BDBF1BDF57
:10130000B0E0B8BBB0E1B7BBB0E0B5BBB0E0B4BBD8
:10131000B0E0B2BBBBEBB1BB2224A0E0B0E02D92A9
:10132000AA31E9F7A0E6B0E00FEF2D920A95E9F7B0
:10133000B1E0B093A2000CDFF3D2B7E0B06CB7B964
:10134000B6B1B460B068B6B90091CA000093AD0000
:10135000B1E0B0936A00F89470D97AD96AD97BD990
:1013600068D97CD966D9F8940AEF1AEFA0B396FF32
:10137000A095A2FF1FC01A95C9F70A95B1F7E0E042
:10138000FCE1B591B43E39F4B591B03E21F4B5918C
:10139000BF3F09F40CC0E0E0F395F395B591B83F79
:1013A00049F4B591B43931F4B591BA3A19F4EE274C
:1013B000F695099413DF2CDF5ADF5ADF0091CA003B
:1013C0000093AD00B8DEB2E0B3BFB2E0BEBDB2E0A4
:1013D000B5BDB1E5B8BFB9BFB0B7B77FB0BFB8B1A1
:1013E000B0B7B860B0BF1FD97894E5DA209270002A
:1013F000B3E096FFB2E0B5BFB0E4BBBFBB27B064BB
:10140000BABF8D7F1AD9626033E02CE0B0919500AD
:10141000BB2321F42CE03A9509F4A5CF0AD980FF2B
:10142000A2CF8E7FB0919600B23078F3B92FBF7102
:101430000091980000939700B0939800B01729F797
:101440002A9521F76D7FB3E096FFB2E0B5BFBB27C9
:10145000B064BABF8D7FB091D400BB2321F4806209
:10146000B92FB0709B2F8F7B20926700E4D885FF47
:1014700005C0B0916700BA3008F08064D6D802E0A9
:1014800085FF01C000E0B0919600B017B8F3F89462
:10149000DFD8DED8DDD87894D0D820928600B091FD
:1014A000BA00B33009F473C0C0D8B091BE00B130F7
:1014B00008F46DC0B0916A00B13008F468C085FDD1
:1014C00018C0B0919600BF3F08F461C0F894C9D825
:1014D0007894B1D8B0919600B130C0F7F894B8D8EC
:1014E000A6D8B6D87894A7D8B0919600BF3FB0F3ED
:1014F000D8C2B3E09B2E9068F894BADE78949BD85B
:10150000F8949F77B5DE80909600B0919600BF3733
:10151000789408F444C087D8F894A3D878949A941F
:1015200051F7C3DEB82DB093C90087D8F89425D2FF
:101530008BD27894BAE09B2E9068F89499DE7894D8
:101540007AD8F8949F7794DE80909600B0919600B8
:10155000BF37789478F767D8F8947AD868D878D86D
:1015600078949A9449F7A1DEB82DBB5FB093C80078
:1015700064D8F89402D277D278945DD8F89478DE63
:101580007894B0919600BF3F08F499CF8AC2009139
:101590009600B09186000B1710F0009386004BD890
:1015A00001E0B091BA00B35009F405E0B0919600A3
:1015B000B01708F074CFF89454D853D852D8789410
:1015C0003CD820926A0020926B0020926C00B0916F
:1015D0006B00B395B0936B00BF3F71F5B0916C0099
:1015E000B395B0936C00B091CC0009E1BA9559F075
:1015F00002E3BA9541F00DE7BA9529F00AEFBA95E2
:1016000011F020926C00B0916C00B017A8F093DD3F
:101610000AD8B0916C00BA95B0936C0020926B0020
:10162000B091CB00B093AD00F8941BD87894B091F2
:10163000CA00B093AD00FFD7FAD7B0916800BB23C2
:1016400019F485FF01C08FCE01E085FD01C006E0E1
:10165000B0919600B01708F4BACFB091BA00B35069
:1016600009F0E9D7B0916800BB2309F47CCEF89467
:1016700062DD209261002092620020926300522C71
:10168000209264002092A1007894B091B700BB0F23
:10169000B0939F0020927E0020927F0020928000D5
:1016A00020928100209282002092AA0060E070E0E7
:1016B00020927100B8E0B093AA007061B4D7B7E08F
:1016C00074FDB7E0B06CB7B9B6B1B068B064B6B984
:1016D000B6B1B6FDFDCF04B115B1B6B1BF77B6B99D
:1016E000112309F00FEF0093AB0067D9B8E0B09376
:1016F000AA00706173DDF894BFEFB0939B00BCD972
:10170000B0916100B0939B00B0939C00B0939D009A
:101710007894B1E0B0936100B09363005B2EB09316
:101720006400B093A400B0919A00B093A300B0916C
:10173000BA00B33019F49F7D87FD906271607260CA
:1017400020926D00A1DCB7DCB0D9B5D9AED9B3D940
:10175000ACD921DB03D8BBDBEBDBADD915DB66FDF8
:1017600036D877FFE8D877FD16D9B1DBF8DBA3D9F7
:1017700012DB66FD48D8ABDB31DC9DD905DB66FDAD
:101780007CD8A5DB42DC97D906DB66FDA6D89FDBBB
:101790007BDC91D9F9DAB7E074FDB7E0B06CB7B98A
:1017A000B6B1B068B064B6B992DB85DC84D905D92E
:1017B00071FF24C0B0919E00B0939B00B0939C0039
:1017C000B0919A00B093A300B1E0B093A40018E1E7
:1017D0002CE0B0916D00B11758F07D7F74602093BC
:1017E0006F00B0919E00B0939B00B0939D0006C027
:1017F000B0919600B13008F0ACCF60C072FF11C05C
:1018000067FD0FC0B0916F00BA9519F47B7F7860C7
:10181000A0CFB0936F00B0919600B13008F099CF8F
:101820004DC020927000B09199000AEF1091D6003F
:10183000112309F003E0B01708F040C085FF04C091
:10184000B0916800BB23D1F1B091BA00B33081F4FC
:1018500095FD03C087FD04C00BC087FF01C008C011
:1018600067FD06C06068B0919E00B0939B0086CF74
:1018700000EF67FF05C0B0919E00B0939B0000E2AF
:10188000B0917B00B01708F464CF67FF17C06F7783
:101890009F7D87FD90627460B2E1B0936F00B0915C
:1018A0009E00B0939B0055CFB0917000B395B0935C
:1018B0007000B0919600BB2309F002C02092700026
:1018C000F89439DC8090B900B2E0B093B90086DCBE
:1018D0008092B90020926100209262002092630001
:1018E000522C2092640020929F0060E070E0789477
:1018F000A2D621DC0091D600002319F0919A909A8B
:10190000939AB7E0B06CB7B9B6B1B460B068B6B985
:1019100085FF05C0B0917000B43008F024CD53CEDF
:10192000EDE0F0E023D0053509F01BC0EEE0F0E07B
:101930001DD00A3A09F015C03AE0A2EBB0E0E3E0AE
:10194000F0E014D00D9331963A95D9F739E1AEEB2A
:10195000B0E0EFE0F0E00AD00D9331963A95D9F778
:1019600002C0F6DB0AD0E8E2F0E00895E199FECF8C
:10197000EEBBFFBBE09A0DB308951ED03AE0A2EB98
:10198000B0E0E3E0F0E00D910FD031963A95D9F751
:1019900039E1AEEBB0E0EFE0F0E00D9105D031962B
:1019A0003A95D9F712D00895E199FECF0DBBEEBB61
:1019B000FFBBE29AE19A0895EDE0F0E00FEFF4DF6B
:1019C000EEE0F0E00FEFF0DF0895EDE0F0E005E588
:1019D000EBDFEEE0F0E00AEAE7DF08953091AE00D9
:1019E0000091AF00313011F40093B200323011F4A5
:1019F0000093B300333011F40093B400343011F489
:101A00000093B600353011F40093B800363011F46D
:101A10000093C400373011F40093B900383011F44A
:101A20000093D500393011F40093CE003A3011F410
:101A30000093BA003B3011F40093BB00089525E0F9
:101A4000FCD52A95E9F7089503D605D607D609D619
:101A5000EED5FED500D602D604D6E9D5F9D5FBD50C
:101A6000FDD5FFD50895FDD5F9D5F5D5F1D5DFD54F
:101A7000F8D5F4D5F0D5ECD5DAD5F3D5EFD5EBD54F
:101A8000E7D508958090AE009090AF00E1D5E0D505
:101A9000DFD5CDD58A94D1F7E4D5C9D59A94E1F7AD
:101AA0000895F894D1DF7894CADFC9DFB1E0B0932C
:101AB000AE00B1E0B093AF002092B000F894E2DF46
:101AC0007894B5E06B2E70909600B7D5B0919600E3
:101AD0007B16C9F7B13018F0BF3F40F107C07EDF79
:101AE000F8944BDFB1DFB8E0B1BDA9DF6A9459F7D4
:101AF000B091B000B395B093B000B33008F4DECF2E
:101B00009EDFB091AF00B395B093AF00F894B09161
:101B1000AE00BA95EEE3F0E0EB0FF21D049178947D
:101B20000395B091AF00B01708F4C6CF88DF87DF08
:101B3000B091AE00B395B093AE00B091AE00BC30A2
:101B400008F4B7CF05DBF89418DFB8E0B1BD77DF54
:021B5000C3CB05
:00000001FF
